:1000000010C017C016C015C014C013C012C011C054
:1000100010C00FC00EC00DC00CC00BC00AC009C07C
:1000200008C011241FBECFE5D1E0DEBFCDBF87D011
:100030009CC0E6CFFC019081862F80959823908309
:10004000ADEFB1E01197F1F700C00000908140FFE3
:1000500002C0962B01C098239083ADEFB1E01197B9
:10006000F1F700C00000908141FF02C0962B01C053
:1000700098239083ADEFB1E01197F1F700C0000035
:10008000908142FF02C0962B01C098239083ADEF70
:10009000B1E01197F1F700C00000908143FF02C06A
:1000A000962B01C098239083ADEFB1E01197F1F743
:1000B00000C00000908144FF02C0962B01C098232D
:1000C0009083ADEFB1E01197F1F700C0000090818F
:1000D00045FF02C0962B01C098239083ADEFB1E09D
:1000E0001197F1F700C00000908146FF02C0962BE7
:1000F00001C098239083ADEFB1E01197F1F700C0F4
:10010000000047FF03C08081862B02C090818923B5
:1001100080838DEF91E00197F1F700C000008081AE
:10012000682B6083ADEFB1E01197F1F700C00000DC
:100130008DEF91E00197F1F700C00000089580E88D
:1001400086BD16BCD99AD19AC29ABA98B299FECFF6
:1001500044E662E08BE390E06DDFB29BFECF45E7C3
:0E01600062E08BE390E066DFF1CFF894FFCF12
:00000001FF
